:1000000012C019C018C017C016C015C014C013C044
:1000100012C011C010C00FC00EC00DC00CC00BC06C
:100020000AC009C008C011241FBECFE5D4E0DEBF5E
:10003000CDBF26D02BC0E4CF89B990BD86E880BD66
:1000400088E18AB908955D9BFECF8CB908955F9BC6
:10005000FECF8CB10895982F92959F709A3010F42E
:10006000905D01C0995C5D9BFECF9CB98F708A301A
:1000700010F4805D01C0895C5D9BFECF8CB9089552
:1000800083E390E0D9DF8AE5DEDFFFCFF894FFCF8E
:00000001FF
